:020000040000FA
:0A00000000000000A4EF01F0B9D1E8
:0800180019EF02F09EA8FED7CB
:10002000AD6E12000E6A0D6EFF0E0D260E2200D070
:10003000D8A01200030E0A6EE60E02D8F5D70A6A9F
:10004000FE0F096EE86A0A5AD8A0120000000906DD
:1000500000D0F8D7800E211A20501C5C256E11E2CA
:10006000256C1C5020C01CF0206E1D5021C01DF0BE
:10007000216E1E5022C01EF0226E1F5023C01FF0A2
:10008000236E1A0E256074D0205272E0246A1D502F
:10009000286E2118276E1D8E218E080E255E08E31E
:1000A00023C024F022C023F021C022F0216AF5D71A
:1000B000252607E0D8902132223223322432252E01
:1000C000F9D727AE33D023501F5E22501E5A21503D
:1000D0001D5A07E2D880000E1F561E561D56800E70
:1000E000281A246C04E01F06000E1E5A1D5A040E26
:1000F000256E1D660DD01EC01DF01FC01EF024C051
:100100001FF0246A080E1C5E29E3252EF2D726D0A4
:100110001DBE08D0D89024361F361E361D361C2E24
:10012000F7D71CD024AE22D0246A0FD023501F262C
:1001300022501E2221501D2206E31D321E321F3284
:1001400024321C4A0DD024AE11D01F3E0FD01E3ECB
:100150000DD01D3E0BD0D8801F90EFD71C6A02D067
:1001600026821C681F6A1E6A800E1D6E28AE1D9EA8
:100170001F5012001D501B6E2118276E1C50D8A452
:1001800020503AE01C267E0E03E31C5E03E336D0CB
:100190001C5E31E31FC019F01EC01AF01B8E218EA9
:1001A0001F6A1E6A1D6A180E286E1B321A32193217
:1001B00006E323501F2622501E2221501D221D32ED
:1001C0001E321F32282EF1D71DBE07D01F361E3615
:1001D0001D361C5210E01C061B3416E31F3E14D0C3
:1001E0001E3E12D01D3E10D0D8801D321E321F324E
:1001F0001C3E0AD003D026841C6A02D026821C68CA
:100200001F6A1E6A800E1D6E27AE1D9E1F501200B3
:100210001CC028F01D501FC01DF01F6E1F36283255
:100220001F32266A1F36283602E32684267E06E120
:100230002680286A1F6A1E6A1D6A0BD0282803E0E0
:10024000D8801F3206D0D8901F3202E1268201D01A
:10025000268626B604D026A20FD026B407D07F0E5D
:100260001F6EFF0E1E6E1D6E1C6E23D0800E1F6E45
:1002700001D01F6A000EF6D726B0FBD71C6A9F0E6E
:100280002860EBD77E0E2864F4D79E0E285C07E02A
:10029000D8901F321E321D321C32282AF6D726A4CF
:1002A00008D0D880000E1C561D561E561F561FAE75
:1002B000E0D71C5012001C6E000E1CBEFF0E1D6EFF
:1002C0001E6E1F6E06D01C6E1D6A1E6A1F6A279E58
:1002D0000AD0279E1FAE07D0D880000E1C561D5690
:1002E0001E561F56278E960E286E1F5209E0080EC6
:1002F00028261DC01CF01EC01DF01FC01EF011D00E
:100300001E520FE1080E285E1D5007E1080E285E00
:100310001C5002E11F5010D01C6A1E6E1CC01DF044
:100320001C6A1EBE06D0D8901C361D361E36280606
:10033000F8D727AE1E9E28501CC01FF01C6E1E5002
:100340001DC01EF01D6E1200400E266E006A4F0E7C
:10035000AF6EB06A240EAC6E900EAB6E00010F0E45
:10036000C16E070EB46EC69AC00E926EE00E936E0A
:10037000C00E946E956AE80E966E70D0F2A409D005
:10038000F2942B4A2C2AD6CF29F0D7CF2AF08176A7
:1003900011009EAA19D0060EAB1412E1E2CF50F064
:1003A000E1CF4FF0512A13EECCF05150E126000E70
:1003B000E222AECFE7FF50C0E2FF4FC0E1FF1100E5
:1003C000AE50AE50AB98AB8811005150525C14E067
:1003D000522AEACF0AF0E9CF09F003EECCF05250EE
:1003E000E926000EEA22EF504E6E0AC0EAFF09C06D
:1003F000E9FFD880120004D0E8684E6ED8A0120041
:100400001200516A526A9D8A9F8AF28EF28C120003
:100410009D9A03EECCF0010EF46EF36AF306000E23
:10042000F45AEE6AF450F310F9E1516A526A9D8A67
:100430001200F29EE0CFCCF4D8CFCDF4E8CFCEF4CA
:10044000F28E0001A192B36AB26AF29ECCC4E0FFC0
:10045000CDC4D8FFCEC4E8FFF28E100093968A86F2
:100460000A0E12EC00F093968A96929089909292DE
:100470008992929489949296899692988998929A60
:10048000899A96908D9096928D9296948D94949050
:100490008B9094928B9294948B9494968B96959047
:1004A0008C9095928C92959E8C9E959C8C9C959A06
:1004B0008C9A95988C98949A8B9A94988B989596F8
:1004C0008C9695948C9493908A9093928A9293941C
:1004D0008A9491EC12F0376800EE53F0680EEE68E3
:1004E000E82EFDD7456A4D6A0301C36BC26BC16B31
:1004F000C06BBF6BBE6BBD6BBC6BBB6B3BC147F0D6
:100500003CC148F03BC249F03CC24AF03BC34BF00F
:100510003CC34CF076DF00017BDFCD6AF294F28AB7
:10052000870ED56EB16AA192A082B36AB26AD08EEC
:10053000A292B10EB16E3F500EEC00F0420E0EECE6
:1005400000F0400E0EEC00F0D6CF29F0D7CF2AF005
:100550003CDF4EC031F0B50E315C07E3FE0E315C7E
:1005600001E301D0386AA5EF0CF031AE38D0386A1B
:10057000840E315C05E131C038F039683A682DD01D
:10058000940E315C05E131C038F03B683C6825D001
:10059000A40E315C05E131C038F03D683E681DD0E5
:1005A000B40E315C05E131C038F03F68406815D0C9
:1005B000C40E315C04E131C038F041680ED0D40E75
:1005C000315C04E131C038F0426807D0E40E315CA0
:1005D00004E131C038F043684468A3EF0CF03852AE
:1005E00004E1A5EF0CF0A3EF0CF0840E385CD8A466
:1005F00046EF07F0392804E131C039F044EF07F045
:1006000031C03AF04D52D8A443EF07F00C0E03016D
:10061000C35D0001D8B043EF07F0420E395C27E11B
:10062000898000EEBBF0D8903A34E926000EEA2229
:10063000EECF07F0EFCF08F007502924036E0850E3
:100640002A20046E000E2B20056E000E2C20066E54
:1006500006C056F005C055F004C054F003C053F076
:1006600046800301BB81BF91000143EF07F0430EB9
:10067000395C27E1898200EEBBF0D8903A34E92654
:10068000000EEA22EECF07F0EFCF08F00750292442
:10069000036E08502A20046E000E2B20056E000EFB
:1006A0002C20066E06C05AF005C059F004C058F060
:1006B00003C057F046800301BB83BF93000143EFA3
:1006C00007F0440E395C27E1898400EEBBF0D89036
:1006D0003A34E926000EEA22EECF07F0EFCF08F019
:1006E00007502924036E08502A20046E000E2B2088
:1006F000056E000E2C20066E06C05EF005C05DF093
:1007000004C05CF003C05BF046800301BB85BF956D
:10071000000143EF07F0450E395C27E1898600EEC2
:10072000BBF0D8903A34E926000EEA22EECF07F06B
:10073000EFCF08F007502924036E08502A20046EDA
:10074000000E2B20056E000E2C20066E06C062F0F7
:1007500005C061F004C060F003C05FF04680030193
:10076000BB87BF97000143EF07F0460E395C27E1D6
:10077000898800EEBBF0D8903A34E926000EEA22D0
:10078000EECF07F0EFCF08F007502924036E085092
:100790002A20046E000E2B20056E000E2C20066E03
:1007A00006C066F005C065F004C064F003C063F0E5
:1007B00046800301BB89BF99000143EF07F0470E54
:1007C000395C27E1898A00EEBBF0D8903A34E926FB
:1007D000000EEA22EECF07F0EFCF08F007502924F1
:1007E000036E08502A20046E000E2B20056E000EAA
:1007F0002C20066E06C06AF005C069F004C068F0DF
:1008000003C067F046800301BB8BBF9B000143EF31
:1008100007F0480E395C27E18D8000EEBBF0D890E0
:100820003A34E926000EEA22EECF07F0EFCF08F0C7
:1008300007502924036E08502A20046E000E2B2036
:10084000056E000E2C20066E06C06EF005C06DF021
:1008500004C06CF003C06BF046800301BB8DBF9DEC
:10086000000143EF07F0490E395C27E18D8200EE6D
:10087000BBF0D8903A34E926000EEA22EECF07F01A
:10088000EFCF08F007502924036E08502A20046E89
:10089000000E2B20056E000E2C20066E06C072F096
:1008A00005C071F004C070F003C06FF04680030112
:1008B000BB8FBF9F000143EF07F04A0E395C27E171
:1008C0008D8400EEBBF0D8903A34E926000EEA227F
:1008D000EECF07F0EFCF08F007502924036E085041
:1008E0002A20046E000E2B20056E000E2C20066EB2
:1008F00006C076F005C075F004C074F003C073F054
:1009000046800301BC81C091000143EF07F04B0E0C
:10091000395C27E18B8000EEBBF0D8903A34E926B1
:10092000000EEA22EECF07F0EFCF08F0075029249F
:10093000036E08502A20046E000E2B20056E000E58
:100940002C20066E06C07AF005C079F004C078F05D
:1009500003C077F046800301BC83C093000143EFDE
:1009600007F04C0E395C27E18B8200EEBBF0D8908B
:100970003A34E926000EEA22EECF07F0EFCF08F076
:1009800007502924036E08502A20046E000E2B20E5
:10099000056E000E2C20066E06C07EF005C07DF0B0
:1009A00004C07CF003C07BF046800301BC85C09589
:1009B000000143EF07F04D0E395C27E18B8400EE18
:1009C000BBF0D8903A34E926000EEA22EECF07F0C9
:1009D000EFCF08F007502924036E08502A20046E38
:1009E000000E2B20056E000E2C20066E06C082F035
:1009F00005C081F004C080F003C07FF04680030191
:100A0000BC87C097000143EF07F04E0E395C27E129
:100A10008B8601EEBBF0D8903A34E926000EEA222C
:100A2000EECF07F0EFCF08F007502924036E0850EF
:100A30002A20046E000E2B20056E000E2C20066E60
:100A400006C086F005C085F004C084F003C083F0C2
:100A500046800301BC89C099000143EF07F04F0EA7
:100A6000395C26E18C8001EEBBF0D8903A34E9265F
:100A7000000EEA22EECF07F0EFCF08F0075029244E
:100A8000036E08502A20046E000E2B20056E000E07
:100A90002C20066E06C08AF005C089F004C088F0DC
:100AA00003C087F046800301BC8BC09B0001EBD1E3
:100AB000500E395C26E18C8201EEBBF0D8903A34BE
:100AC000E926000EEA22EECF07F0EFCF08F007503C
:100AD0002924036E08502A20046E000E2B20056E78
:100AE000000E2C20066E06C08EF005C08DF004C0EE
:100AF0008CF003C08BF046800301BC8DC09D0001CB
:100B0000C2D1510E395C26E18C8E01EEBBF0D8903B
:100B10003A34E926000EEA22EECF07F0EFCF08F0D4
:100B200007502924036E08502A20046E000E2B2043
:100B3000056E000E2C20066E06C092F005C091F0E6
:100B400004C090F003C08FF046800301BC8FC09FAB
:100B5000000199D1520E395C26E18C8C02EEBBF07B
:100B6000D8903A34E926000EEA22EECF07F0EFCF14
:100B700008F007502924036E08502A20046E000E46
:100B80002B20056E000E2C20066E06C096F005C0C8
:100B900095F004C094F003C093F046800301BD813A
:100BA000C191000170D1530E395C26E18C8A02EEAE
:100BB000BBF0D8903A34E926000EEA22EECF07F0D7
:100BC000EFCF08F007502924036E08502A20046E46
:100BD000000E2B20056E000E2C20066E06C09AF02B
:100BE00005C099F004C098F003C097F04680030157
:100BF000BD83C193000147D1540E395C26E18C8836
:100C000002EEBBF0D8903A34E926000EEA22EECF8D
:100C100007F0EFCF08F007502924036E08502A2070
:100C2000046E000E2B20056E000E2C20066E06C0F2
:100C30009EF005C09DF004C09CF003C09BF0468070
:100C40000301BD85C19500011ED1550E395C26E119
:100C50008B8A02EEBBF0D8903A34E926000EEA22E5
:100C6000EECF07F0EFCF08F007502924036E0850AD
:100C70002A20046E000E2B20056E000E2C20066E1E
:100C800006C0A2F005C0A1F004C0A0F003C09FF010
:100C900046800301BD87C1970001F5D0560E395C2F
:100CA00026E18B8802EEBBF0D8903A34E926000E9C
:100CB000EA22EECF07F0EFCF08F007502924036EA9
:100CC00008502A20046E000E2B20056E000E2C20EA
:100CD000066E06C0A6F005C0A5F004C0A4F003C0CF
:100CE000A3F046800301BD89C1990001CCD0570E05
:100CF000395C26E18C8602EEBBF0D8903A34E926C6
:100D0000000EEA22EECF07F0EFCF08F007502924BB
:100D1000036E08502A20046E000E2B20056E000E74
:100D20002C20066E06C0AAF005C0A9F004C0A8F0E9
:100D300003C0A7F046800301BD8BC19B0001A3D077
:100D4000580E395C26E18C8402EEBBF0D8903A3420
:100D5000E926000EEA22EECF07F0EFCF08F00750A9
:100D60002924036E08502A20046E000E2B20056EE5
:100D7000000E2C20066E06C0AEF005C0ADF004C01B
:100D8000ACF003C0ABF046800301BD8DC19D0001F6
:100D90007AD0590E395C26E18A8002EEBBF0D890F9
:100DA0003A34E926000EEA22EECF07F0EFCF08F042
:100DB00007502924036E08502A20046E000E2B20B1
:100DC000056E000E2C20066E06C0B2F005C0B1F014
:100DD00004C0B0F003C0AFF046800301BD8FC19FD7
:100DE000000151D05A0E395C26E18A8202EEBBF036
:100DF000D8903A34E926000EEA22EECF07F0EFCF82
:100E000008F007502924036E08502A20046E000EB3
:100E10002B20056E000E2C20066E06C0B6F005C015
:100E2000B5F004C0B4F003C0B3F046800301BE8146
:100E3000C291000128D05B0E395C24E18A8402EE65
:100E4000BBF0D8903A34E926000EEA22EECF07F044
:100E5000EFCF08F007502924036E08502A20046EB3
:100E6000000E2B20056E000E2C20066E06C0BAF078
:100E700005C0B9F004C0B8F003C0B7F04680030164
:100E8000BE83C29300013968A3EF0CF0940E385C66
:100E9000D8A479EF0CF03B2804E131C03BF078EFA7
:100EA0000CF031C03CF03C52D8A477EF0AF04D5220
:100EB000D8A475EF0AF00C0E0301C35D0001D8B091
:100EC00075EF0AF0420E3B5C1CE1898047502924F3
:100ED000036E48502A20046E000E2B20056E000E73
:100EE0002C20066E06C056F005C055F004C054F024
:100EF00003C053F046800301BB81BF91000175EF31
:100F00000AF0430E3B5C1CE1898247502924036EA2
:100F100048502A20046E000E2B20056E000E2C2057
:100F2000066E06C05AF005C059F004C058F003C060
:100F300057F046800301BB83BF93000175EF0AF0B1
:100F4000440E3B5C1CE1898447502924036E4850C1
:100F50002A20046E000E2B20056E000E2C20066E3B
:100F600006C05EF005C05DF004C05CF003C05BF03D
:100F700046800301BB85BF95000175EF0AF0450E61
:100F80003B5C1CE1898647502924036E48502A2087
:100F9000046E000E2B20056E000E2C20066E06C07F
:100FA00062F005C061F004C060F003C05FF04680ED
:100FB0000301BB87BF97000175EF0AF0460E3B5C4B
:100FC0001CE1898847502924036E48502A20046E6A
:100FD000000E2B20056E000E2C20066E06C066F05B
:100FE00005C065F004C064F003C063F046800301EF
:100FF000BB89BF99000175EF0AF0470E3B5C1CE10D
:10100000898A47502924036E48502A20046E000E16
:101010002B20056E000E2C20066E06C06AF005C05F
:1010200069F004C068F003C067F046800301BB8B21
:10103000BF9B000175EF0AF0480E3B5C1CE18D8000
:1010400047502924036E48502A20046E000E2B209E
:10105000056E000E2C20066E06C06EF005C06DF009
:1010600004C06CF003C06BF046800301BB8DBF9DD4
:10107000000175EF0AF0490E3B5C1CE18D82475080
:101080002924036E48502A20046E000E2B20056E82
:10109000000E2C20066E06C072F005C071F004C070
:1010A00070F003C06FF046800301BB8FBF9F00014B
:1010B00075EF0AF04A0E3B5C1BE18D8447502924F2
:1010C000036E48502A20046E000E2B20056E000E81
:1010D0002C20066E06C076F005C075F004C074F0D2
:1010E00003C073F046800301BC81C0910001FDD1B3
:1010F0004B0E3B5C1BE18B8047502924036E48500C
:101100002A20046E000E2B20056E000E2C20066E89
:1011100006C07AF005C079F004C078F003C077F01B
:1011200046800301BC83C0930001DFD14C0E3B5CC1
:101130001BE18B8247502924036E48502A20046EFD
:10114000000E2B20056E000E2C20066E06C07EF0D1
:1011500005C07DF004C07CF003C07BF04680030135
:10116000BC85C0950001C1D14D0E3B5C1BE18B8459
:1011700047502924036E48502A20046E000E2B206D
:10118000056E000E2C20066E06C082F005C081F0B0
:1011900004C080F003C07FF046800301BC87C09785
:1011A0000001A3D14E0E3B5C1BE18B8649502924E4
:1011B000036E4A502A20046E000E2B20056E000E8E
:1011C0002C20066E06C086F005C085F004C084F0B1
:1011D00003C083F046800301BC89C099000185D11A
:1011E0004F0E3B5C1BE18C8049502924036E4A5012
:1011F0002A20046E000E2B20056E000E2C20066E99
:1012000006C08AF005C089F004C088F003C087F0EA
:1012100046800301BC8BC09B000167D1500E3B5C34
:101220001BE18C8249502924036E4A502A20046E07
:10123000000E2B20056E000E2C20066E06C08EF0D0
:1012400005C08DF004C08CF003C08BF04680030114
:10125000BC8DC09D000149D1510E3B5C1BE18C8EC1
:1012600049502924036E4A502A20046E000E2B2078
:10127000056E000E2C20066E06C092F005C091F09F
:1012800004C090F003C08FF046800301BC8FC09F64
:1012900000012BD1520E3B5C1BE18C8C4B5029245E
:1012A000036E4C502A20046E000E2B20056E000E9B
:1012B0002C20066E06C096F005C095F004C094F090
:1012C00003C093F046800301BD81C19100010DD19F
:1012D000530E3B5C1BE18C8A4B502924036E4C500F
:1012E0002A20046E000E2B20056E000E2C20066EA8
:1012F00006C09AF005C099F004C098F003C097F0BA
:1013000046800301BD83C1930001EFD0540E3B5CC6
:101310001BE18C884B502924036E4C502A20046E0C
:10132000000E2B20056E000E2C20066E06C09EF0CF
:1013300005C09DF004C09CF003C09BF046800301F3
:10134000BD85C1950001D1D0550E3B5C1BE18B8A58
:101350004B502924036E4C502A20046E000E2B2083
:10136000056E000E2C20066E06C0A2F005C0A1F08E
:1013700004C0A0F003C09FF046800301BD87C19761
:101380000001B3D0560E3B5C1BE18B884B502924E7
:10139000036E4C502A20046E000E2B20056E000EAA
:1013A0002C20066E06C0A6F005C0A5F004C0A4F06F
:1013B00003C0A3F046800301BD89C199000195D007
:1013C000570E3B5C1BE18C864B502924036E4C501E
:1013D0002A20046E000E2B20056E000E2C20066EB7
:1013E00006C0AAF005C0A9F004C0A8F003C0A7F089
:1013F00046800301BD8BC19B000177D0580E3B5C3A
:101400001BE18C844B502924036E4C502A20046E1F
:10141000000E2B20056E000E2C20066E06C0AEF0CE
:1014200005C0ADF004C0ACF003C0ABF046800301D2
:10143000BD8DC19D000159D0590E3B5C1BE18A80D6
:101440004B502924036E4C502A20046E000E2B2092
:10145000056E000E2C20066E06C0B2F005C0B1F07D
:1014600004C0B0F003C0AFF046800301BD8FC19F40
:1014700000013BD05A0E3B5C1BE18A824B50292471
:10148000036E4C502A20046E000E2B20056E000EB9
:101490002C20066E06C0B6F005C0B5F004C0B4F04E
:1014A00003C0B3F046800301BE81C29100011DD08C
:1014B0005B0E3B5C19E18A844B502924036E4C502F
:1014C0002A20046E000E2B20056E000E2C20066EC6
:1014D00006C0BAF005C0B9F004C0B8F003C0B7F058
:1014E00046800301BE83C293000178EF0CF0420EE8
:1014F0003B5C10E189900301BB31000107E35668B2
:1015000055685468536846800301BB910301BF814D
:101510000001EDD1430E3B5C11E189920301BB5107
:101520000001E8A207D05A68596858685768468091
:101530000301BB930301BF830001D9D1440E3B5C7F
:1015400011E189940301BB510001E8A407D05E6852
:101550005D685C685B6846800301BB950301BF85DD
:101560000001C5D1450E3B5C11E189960301BB51D9
:101570000001E8A607D06268616860685F6846801D
:101580000301BB970301BF870001B1D1460E3B5C4D
:1015900011E189980301BB510001E8A807D06668F2
:1015A00065686468636846800301BB990301BF896D
:1015B00000019DD1470E3B5C11E1899A0301BB51AB
:1015C0000001E8AA07D06A686968686867684680A9
:1015D0000301BB9B0301BF8B000189D1480E3B5C1B
:1015E00011E18D900301BB510001E8AC07D06E689A
:1015F0006D686C686B6846800301BB9D0301BF8DFD
:10160000000175D1490E3B5C10E18D920301BB35A1
:10161000000107E37268716870686F6846800301B3
:10162000BB9F0301BF8F000162D14A0E3B5C10E1FA
:101630008D940301BC31000107E376687568746816
:10164000736846800301BC910301C08100014FD142
:101650004B0E3B5C11E18B900301BC510001E8A2F1
:1016600007D07A6879687868776846800301BC9308
:101670000301C08300013BD14C0E3B5C11E18B9216
:101680000301BC510001E8A407D07E687D687C6836
:101690007B6846800301BC950301C085000127D10A
:1016A0004D0E3B5C11E18B940301BC510001E8A697
:1016B00007D08269816980697F6846800301BC9791
:1016C0000301C087000113D14E0E3B5C11E18B96E4
:1016D0000301BC510001E8A807D0866985698469C7
:1016E000836946800301BC990301C0890001FFD0D2
:1016F0004F0E3B5C11E18C900301BC510001E8AA44
:1017000007D08A6989698869876946800301BC9B1B
:101710000301C08B0001EBD0500E3B5C11E18C92B9
:101720000301BC510001E8AC07D08E698D698C695A
:101730008B6946800301BC9D0301C08D0001D7D099
:10174000510E3B5C10E18C9E0301BC35000107E3A8
:101750009269916990698F6946800301BC9F03017A
:10176000C08F0001C4D0520E3B5C10E18C9C030181
:10177000BD31000107E396699569946993694680D4
:101780000301BD910301C1810001B1D0530E3B5C47
:1017900011E18C9A0301BD510001E8A207D09A69BA
:1017A00099699869976946800301BD930301C183D4
:1017B00000019DD0540E3B5C11E18C980301BD519A
:1017C0000001E8A407D09E699D699C699B694680D9
:1017D0000301BD950301C185000189D0550E3B5C15
:1017E00011E18B9A0301BD510001E8A607D0A2695F
:1017F000A169A0699F6946800301BD970301C18764
:10180000000175D0560E3B5C11E18B980301BD5170
:101810000001E8A807D0A669A569A469A369468064
:101820000301BD990301C189000161D0570E3B5CE2
:1018300011E18C960301BD510001E8AA07D0AA6905
:10184000A969A869A76946800301BD9B0301C18BF3
:1018500000014DD0580E3B5C11E18C940301BD5149
:101860000001E8AC07D0AE69AD69AC69AB694680F0
:101870000301BD9D0301C18D000139D0590E3B5CB0
:1018800010E18A900301BD35000107E3B269B16937
:10189000B069AF6946800301BD9F0301C18F00019C
:1018A00026D05A0E3B5C10E18A920301BE31000142
:1018B00007E3B669B569B469B36946800301BE91AF
:1018C0000301C281000113D05B0E3B5C0FE18A94DF
:1018D0000301BE510001E8A207D0BA69B969B8692D
:1018E000B76946800301BE930301C28300013B68D0
:1018F0002AD0A40E385C0AE13D2803E131C03DF056
:1019000003D031C03EF0D0D920D01DD0B40E385C09
:1019100009E13F2803E131C03FF003D031C040F07E
:10192000CBD911D0C40E385C06E1412803E131C0A7
:1019300041F0BCD908D0D40E385C05E1422803E15F
:1019400031C042F0B7D946B058D91A0E375CD8B07A
:1019500045D13350295C34502A5835502B583650D5
:101960002C58D8A03AD1368E375209E18990566862
:101970005568546853680301BB9100012DD1010ED5
:10198000375C09E189925A685968586857680301B9
:10199000BB93000121D1020E375C09E189945E6896
:1019A0005D685C685B680301BB95000115D1030E9F
:1019B000375C09E189966268616860685F68030165
:1019C000BB97000109D1040E375C09E1899866686C
:1019D0006568646863680301BB990001FDD0050E6A
:1019E000375C09E1899A6A68696868686768030111
:1019F000BB9B0001F1D0060E375C09E18D906E684B
:101A00006D686C686B680301BB9D0001E5D0070E33
:101A1000375C09E18D927268716870686F680301C4
:101A2000BB9F0001D9D0080E375C09E18D94766820
:101A30007568746873680301BC910001CDD0090E0C
:101A4000375C09E18B907A68796878687768030178
:101A5000BC930001C1D00A0E375C09E18B927E680D
:101A60007D687C687B680301BC950001B5D00B0ED6
:101A7000375C09E18B948269816980697F68030121
:101A8000BC970001A9D00C0E375C09E18B968669E2
:101A90008569846983690301BC9900019DD00D0E9D
:101AA000375C09E18C908A698969886987690301D3
:101AB000BC9B000191D00E0E375C09E18C928E69BF
:101AC0008D698C698B690301BC9D000185D00F0E67
:101AD000375C09E18C9E9269916990698F69030175
:101AE000BC9F000179D0100E375C09E18C9C96698F
:101AF0009569946993690301BD9100016DD0110E40
:101B0000375C09E18C9A9A69996998699769030128
:101B1000BD93000161D0120E375C09E18C989E697B
:101B20009D699C699B690301BD95000155D0130E09
:101B3000375C09E18B9AA269A169A0699F690301D9
:101B4000BD97000149D0140E375C09E18B98A66956
:101B5000A569A469A3690301BD9900013DD0150ED3
:101B6000375C09E18C96AA69A969A869A76903018C
:101B7000BD9B000131D0160E375C09E18C94AE6933
:101B8000AD69AC69AB690301BD9D000125D0170E9D
:101B9000375C09E18A90B269B169B069AF69030144
:101BA000BD9F000119D0180E375C09E18A92B66911
:101BB000B569B469B3690301BE9100010DD0190E76
:101BC000375C09E18A94BA69B969B869B7690301F0
:101BD000BE93000101D00ED010D80CD02CAE0AD08C
:101BE0002C6A2B6A2A6A296A00EE53F0680EEE68A6
:101BF000E82EFDD78178A4EF02F03768368E030116
:101C0000C36B326A00011A0E325CD8B04BD0D89048
:101C10003234E96EEA6AEA36E936EA36530EE926E4
:101C2000000EEA22EFCF03F0ECCF04F0ECCF05F08A
:101C3000ECCF06F03350035C34500458355005584F
:101C40003650065815E2D8903234E96EEA6AEA3620
:101C5000E936EA36530EE926000EEA22EFCF33F0DA
:101C6000ECCF34F0ECCF35F0ECCF36F032C037F0BB
:101C7000BEC30CF0BDC30BF0BCC30AF0BBC309F07C
:101C80003250E82A0C320B320A320932E82EFAD7E7
:101C9000010ED8A0000E036E0301C3270001322AF3
:101CA000D8A0B0D7469012003D68120041681200DB
:101CB0004368120042681200190E3F5C23E100EEF7
:101CC000BBF0D8904034E926000EEA22EECF47F070
:101CD000EFCF48F001EEBBF0D8904034E926000E7B
:101CE000EA22EECF49F0EFCF4AF002EEBBF0D890F7
:101CF0004034E926000EEA22EECF4BF0EFCF4CF055
:101D00003CEF12F0400E3F5C08E1405202E14D6AA8
:101D100002D0010E4D6E3CEF12F0420E3F5C16E118
:101D2000405204E145903EEC12F00ED04D6A3BC1AA
:101D300047F03CC148F03BC249F03CC24AF03BC3CB
:101D40004BF03CC34CF045803CEF12F07B0E3F5C07
:101D5000D8A43CEF12F04D52D8A43BEF12F003018F
:101D6000BF3100011EE30C0E0301C35D000119E247
:101D7000898047502924036E48502A20046E000EA3
:101D80002B20056E000E2C20066E06C056F005C0F6
:101D900055F004C054F003C053F046800301BB81EA
:101DA000C32B0301BF510001E8A21ED00C0E03019A
:101DB000C35D000119E2898247502924036E48500F
:101DC0002A20046E000E2B20056E000E2C20066EBD
:101DD00006C05AF005C059F004C058F003C057F0CF
:101DE00046800301BB83C32B0301BF510001E8A45C
:101DF0001ED00C0E0301C35D000119E28984475017
:101E00002924036E48502A20046E000E2B20056EF4
:101E1000000E2C20066E06C05EF005C05DF004C00A
:101E20005CF003C05BF046800301BB85C32B03015C
:101E3000BF510001E8A61ED00C0E0301C35D0001D6
:101E400019E2898647502924036E48502A20046EDF
:101E5000000E2B20056E000E2C20066E06C062F0D0
:101E600005C061F004C060F003C05FF0468003016C
:101E7000BB87C32B0301BF510001E8A81ED00C0E85
:101E80000301C35D000119E2898847502924036ECC
:101E900048502A20046E000E2B20056E000E2C20C8
:101EA000066E06C066F005C065F004C064F003C0AD
:101EB00063F046800301BB89C32B0301BF510001BE
:101EC000E8AA1ED00C0E0301C35D000119E2898A45
:101ED00047502924036E48502A20046E000E2B2000
:101EE000056E000E2C20066E06C06AF005C069F073
:101EF00004C068F003C067F046800301BB8BC32BAE
:101F00000301BF510001E8AC1ED00C0E0301C35DFC
:101F1000000119E28D8047502924036E48502A2081
:101F2000046E000E2B20056E000E2C20066E06C0DF
:101F30006EF005C06DF004C06CF003C06BF046801D
:101F40000301BB8DC32B0301BF3500011EE30C0E43
:101F50000301C35D000119E28D8247502924036EFD
:101F600048502A20046E000E2B20056E000E2C20F7
:101F7000066E06C072F005C071F004C070F003C0B8
:101F80006FF046800301BB8FC32B0301C0310001FA
:101F90001EE30C0E0301C35D000119E28D8447505E
:101FA0002924036E48502A20046E000E2B20056E53
:101FB000000E2C20066E06C076F005C075F004C039
:101FC00074F003C073F046800301BC81C32B03018E
:101FD000C0510001E8A21ED00C0E0301C35D000138
:101FE00019E28B8047502924036E48502A20046E42
:101FF000000E2B20056E000E2C20066E06C07AF017
:1020000005C079F004C078F003C077F04680030182
:10201000BC83C32B0301C0510001E8A41ED00C0EE9
:102020000301C35D000119E28B8247502924036E2E
:1020300048502A20046E000E2B20056E000E2C2026
:10204000066E06C07EF005C07DF004C07CF003C0C3
:102050007BF046800301BC85C32B0301C051000106
:10206000E8A61ED00C0E0301C35D000119E28B84AB
:1020700047502924036E48502A20046E000E2B205E
:10208000056E000E2C20066E06C082F005C081F0A1
:1020900004C080F003C07FF046800301BC87C32BDF
:1020A0000301C0510001E8A81ED00C0E0301C35D5E
:1020B000000119E28B8649502924036E4A502A20D8
:1020C000046E000E2B20056E000E2C20066E06C03E
:1020D00086F005C085F004C084F003C083F046801C
:1020E0000301BC89C32B0301C0510001E8AA1ED023
:1020F0000C0E0301C35D000119E28C8049502924B4
:10210000036E4A502A20046E000E2B20056E000E2E
:102110002C20066E06C08AF005C089F004C088F045
:1021200003C087F046800301BC8BC32B0301C05161
:102130000001E8AC1ED00C0E0301C35D000119E2E2
:102140008C8249502924036E4A502A20046E000EC6
:102150002B20056E000E2C20066E06C08EF005C0EA
:102160008DF004C08CF003C08BF046800301BC8D61
:10217000C32B0301C03500011EE30C0E0301C35D38
:10218000000119E28C8E49502924036E4A502A20FE
:10219000046E000E2B20056E000E2C20066E06C06D
:1021A00092F005C091F004C090F003C08FF046801B
:1021B0000301BC8FC32B0301C13100011EE30C0ED0
:1021C0000301C35D000119E28C8C4B502924036E7E
:1021D0004C502A20046E000E2B20056E000E2C2081
:1021E000066E06C096F005C095F004C094F003C0DA
:1021F00093F046800301BD81C32B0301C15100014F
:10220000E8A21ED00C0E0301C35D000119E28C8A06
:102210004B502924036E4C502A20046E000E2B20B4
:10222000056E000E2C20066E06C09AF005C099F0CF
:1022300004C098F003C097F046800301BD83C32B10
:102240000301C1510001E8A41ED00C0E0301C35DBF
:10225000000119E28C884B502924036E4C502A202F
:10226000046E000E2B20056E000E2C20066E06C09C
:102270009EF005C09DF004C09CF003C09BF046801A
:102280000301BD85C32B0301C1510001E8A61ED087
:102290000C0E0301C35D000119E28B8A4B50292407
:1022A000036E4C502A20046E000E2B20056E000E8B
:1022B0002C20066E06C0A2F005C0A1F004C0A0F05C
:1022C00003C09FF046800301BD87C32B0301C151AA
:1022D0000001E8A81ED00C0E0301C35D000119E245
:1022E0008B884B502924036E4C502A20046E000E1C
:1022F0002B20056E000E2C20066E06C0A6F005C031
:10230000A5F004C0A4F003C0A3F046800301BD897A
:10231000C32B0301C1510001E8AA1ED00C0E03011A
:10232000C35D000119E28C864B502924036E4C508A
:102330002A20046E000E2B20056E000E2C20066E47
:1023400006C0AAF005C0A9F004C0A8F003C0A7F019
:1023500046800301BD8BC32B0301C1510001E8ACD2
:102360001ED00C0E0301C35D000119E28C844B509A
:102370002924036E4C502A20046E000E2B20056E7B
:10238000000E2C20066E06C0AEF005C0ADF004C0F5
:10239000ACF003C0ABF046800301BD8DC32B03013D
:1023A000C13500011EE30C0E0301C35D000119E2FB
:1023B0008A804B502924036E4C502A20046E000E54
:1023C0002B20056E000E2C20066E06C0B2F005C054
:1023D000B1F004C0B0F003C0AFF046800301BD8F80
:1023E000C32B0301C23100011EE30C0E0301C35DC8
:1023F000000119E28A824B502924036E4C502A2096
:10240000046E000E2B20056E000E2C20066E06C0FA
:10241000B6F005C0B5F004C0B4F003C0B3F0468018
:102420000301BE81C32B0301C2510001E8A21ED0EB
:102430000C0E0301C35D000119E28A844B5029246C
:10244000036E4C502A20046E000E2B20056E000EE9
:102450002C20066E06C0BAF005C0B9F004C0B8F072
:1024600003C0B7F046800301BE83C32B0301C26BD8
:10247000C16BC06BBF6B00013F68120000EE53F0F0
:10248000680EEE68E82EFDD792908990929289921C
:10249000929489949296899692988998929A899A18
:1024A00096908D9096928D9296948D9494908B9018
:1024B00094928B9294948B9494968B9695908C9006
:1024C00095928C92959E8C9E959C8C9C959A8C9ABC
:1024D00095988C98949A8B9A94988B9895968C96BC
:1024E00095948C9493908A9093928A9293948A94E0
:1024F0004D6A0301BE6BBD6BBC6BBB6BC26BC16B2A
:10250000C06BBF6BC36B3BC147F03CC148F03BC2E3
:1025100049F03CC24AF03BC34BF03CC34CF00001D5
:102520001200BC6BBB6B090EBE6FEF0EBD6F0F0EC2
:1025300001013C6F2F0E3B6F140EBA6F450EB96F41
:102540003BC103F03CC104F0BDC007F0BEC008F0C1
:102550000750035C1C6E085004581D6E65EC01F0BA
:102560001FC014F01EC013F01DC012F01CC011F0EB
:1025700014C0CBF313C0CAF312C0C9F3060E115C2A
:1025800002E22684000E0301C86F020E326E0001C3
:10259000400E325CD8B049D0325063EC01F0CBC36E
:1025A00023F0CAC322F0C9C321F0C8C320F0BAEC9B
:1025B00000F01FC014F01EC013F01DC012F01CC0AC
:1025C00011F0BDC003F0BEC004F003C01CF004C095
:1025D0001DF065EC01F014C023F013C022F012C00E
:1025E00021F011C020F02CEC00F01FC0C7F31EC07A
:1025F000C6F31DC0C5F31CC0C4F3C7C31FF0C6C3D8
:102600001EF0C5C31DF0C4C31CF008EC01F000EEC1
:10261000BBF0D8903234E926000EEA221CC0EEFF4F
:102620001DC0EFFF322AD8A0B2D7B9C103F0BAC19A
:1026300004F03BC107F03CC108F00750035C1C6E7E
:10264000085004581D6E65EC01F01FC014F01EC048
:1026500013F01DC012F01CC011F014C0CBF313C056
:10266000CAF312C0C9F3060E115C02E22684000E02
:102670000301C86F410E326E00017F0E325CD8B08C
:1026800078D0CBC314F0CAC313F0C9C312F0C8C3C7
:1026900011F032505BEC01F01FC018F01EC017F0B3
:1026A0001DC016F01CC015F0236A226A216A850E2F
:1026B000206E18C01FF017C01EF016C01DF015C008
:1026C0001CF02AEC00F01FC018F01EC017F01DC04F
:1026D00016F01CC015F014C023F013C022F012C075
:1026E00021F011C020F018C01FF017C01EF016C056
:1026F0001DF015C01CF0BAEC00F01FC014F01EC095
:1027000013F01DC012F01CC011F03BC103F03CC11E
:1027100004F003C01CF004C01DF065EC01F014C00F
:1027200023F013C022F012C021F011C020F02CECD5
:1027300000F01FC0C7F31EC0C6F31DC0C5F31CC008
:10274000C4F3C7C31FF0C6C31EF0C5C31DF0C4C386
:102750001CF008EC01F000EEBBF0D8903234E92612
:10276000000EEA221CC0EEFF1DC0EFFF322AD8A0E7
:1027700083D70101BC6BBB6B010EBE6F220EBD6F18
:102780000C0E02013C6F650E3B6F130EBA6FEC0E20
:10279000B96F3BC203F03CC204F0BDC107F0BEC13B
:1027A00008F00750035C1C6E085004581D6E65EC61
:1027B00001F01FC014F01EC013F01DC012F01CC0A9
:1027C00011F014C0CBF313C0CAF312C0C9F3060E44
:1027D000115C02E22684000E0301C86F020E326E05
:1027E0000001400E325CD8B049D0325063EC01F0A9
:1027F000CBC323F0CAC322F0C9C321F0C8C320F061
:10280000BAEC00F01FC014F01EC013F01DC012F08F
:102810001CC011F0BDC103F0BEC104F003C01CF028
:1028200004C01DF065EC01F014C023F013C022F0C9
:1028300012C021F011C020F02CEC00F01FC0C7F333
:102840001EC0C6F31DC0C5F31CC0C4F3C7C31FF030
:10285000C6C31EF0C5C31DF0C4C31CF008EC01F0D4
:1028600001EEBBF0D8903234E926000EEA221CC0FB
:10287000EEFF1DC0EFFF322AD8A0B2D7B9C203F0D5
:10288000BAC204F03BC207F03CC208F00750035C38
:102890001C6E085004581D6E65EC01F01FC014F04A
:1028A0001EC013F01DC012F01CC011F014C0CBF3F9
:1028B00013C0CAF312C0C9F3060E115C02E22684EB
:1028C000000E0301C86F410E326E00017F0E325CB4
:1028D000D8B078D0CBC314F0CAC313F0C9C312F078
:1028E000C8C311F032505BEC01F01FC018F01EC0DD
:1028F00017F01DC016F01CC015F0236A226A216A69
:10290000850E206E18C01FF017C01EF016C01DF0F7
:1029100015C01CF02AEC00F01FC018F01EC017F004
:102920001DC016F01CC015F014C023F013C022F017
:1029300012C021F011C020F018C01FF017C01EF007
:1029400016C01DF015C01CF0BAEC00F01FC014F04A
:102950001EC013F01DC012F01CC011F03BC203F0EA
:102960003CC204F003C01CF004C01DF065EC01F093
:1029700014C023F013C022F012C021F011C020F0C7
:102980002CEC00F01FC0C7F31EC0C6F31DC0C5F37A
:102990001CC0C4F3C7C31FF0C6C31EF0C5C31DF0DF
:1029A000C4C31CF008EC01F001EEBBF0D890323447
:1029B000E926000EEA221CC0EEFF1DC0EFFF322AFE
:1029C000D8A083D70201BC6BBB6B010EBE6F220E79
:1029D000BD6F0A0E03013C6FDA0E3B6F140EBA6F27
:1029E000450EB96F3BC303F03CC304F0BDC207F012
:1029F000BEC208F00750035C1C6E085004581D6EE0
:102A000065EC01F01FC014F01EC013F01DC012F0E1
:102A10001CC011F014C0CBF313C0CAF312C0C9F329
:102A2000060E115C02E22684000E0301C86F020E3E
:102A3000326E0001400E325CD8B049D0325063ECA7
:102A400001F0CBC323F0CAC322F0C9C321F0C8C32D
:102A500020F0BAEC00F01FC014F01EC013F01DC02F
:102A600012F01CC011F0BDC203F0BEC204F003C0DE
:102A70001CF004C01DF065EC01F014C023F013C07D
:102A800022F012C021F011C020F02CEC00F01FC089
:102A9000C7F31EC0C6F31DC0C5F31CC0C4F3C7C333
:102AA0001FF0C6C31EF0C5C31DF0C4C31CF008EC64
:102AB00001F002EEBBF0D8903234E926000EEA2293
:102AC0001CC0EEFF1DC0EFFF322AD8A0B2D7B9C399
:102AD00003F0BAC304F03BC307F03CC308F007504F
:102AE000035C1C6E085004581D6E65EC01F01FC09D
:102AF00014F01EC013F01DC012F01CC011F014C061
:102B0000CBF313C0CAF312C0C9F3060E115C02E284
:102B10002684000E0301C86F410E326E00017F0E45
:102B2000325CD8B078D0CBC314F0CAC313F0C9C399
:102B300012F0C8C311F032505BEC01F01FC018F066
:102B40001EC017F01DC016F01CC015F0236A226AC3
:102B5000216A850E206E18C01FF017C01EF016C027
:102B60001DF015C01CF02AEC00F01FC018F01EC0AC
:102B700017F01DC016F01CC015F014C023F013C0D0
:102B800022F012C021F011C020F018C01FF017C0B1
:102B90001EF016C01DF015C01CF0BAEC00F01FC0EE
:102BA00014F01EC013F01DC012F01CC011F03BC386
:102BB00003F03CC304F003C01CF004C01DF065EC3E
:102BC00001F014C023F013C022F012C021F011C094
:102BD00020F02CEC00F01FC0C7F31EC0C6F31DC0D0
:102BE000C5F31CC0C4F3C7C31FF0C6C31EF0C5C3E2
:102BF0001DF0C4C31CF008EC01F002EEBBF0D8904D
:102C00003234E926000EEA221CC0EEFF1DC0EFFFA1
:0A2C1000322AD8A083D71200FFD7A4
:020000040030CA
:0300010006160ED2
:020005008580F4
:060008000FC00FE00F40E5
:00000001FF
